:04000000B601DD293F
:10000800B616B61EB612B6190D28B6154620031830
:1000180034280830A3005A20A20DA30B0F28B61EBF
:100028003F2064206020B61A3420392022080310AB
:10003800D829B616B61EB61236192728FE39B700C3
:1000480036150310D829361A2F28A600361646204A
:100058000318342826084D2003183428B61ED8293A
:100068003F20642036113612B6113A088400380849
:100078008417800445283A088400380980058417C5
:1000880080050800392064203F2060203708B61911
:100098000138A2000830A300A20D03183920031C60
:1000A8003F2064206020A30B5028392064203A08A0
:1000B800840038080005FF3E3B08840039094228BF
:1000C8003B08840039083C280408A6003A08840044
:1000D8008030B7050830A70003100318B70A82203C
:1000E800A60CA70B71280000AB1A370C8220DB2165
:1000F800031482202F08A3002E0841298413AB1F64
:100108009128000838042B1F38068000841700083F
:100118003804031C380680009C2800083804031C97
:1001280038062B1B380680008417380980059C2860
:100138002B081F39003EA1002A08083E0318A10A0F
:1001480000004E29B71329080319B7170430A8006F
:10015800250EB3202508B320240EB32024080F3918
:10016800F63E0318073E0A3ED628B7132908031996
:10017800B7170530A8002730A3001030CF20033070
:10018800A300E830CF20A3016430CF20A3010A30B8
:10019800CF202408D628A2002508A1002408A00002
:1001A800A1212008A000A8030319B71329080319DF
:1001B800E0282802031808002008031DB713B71BFE
:1001C8000800303ED3290830A600A7003B08840069
:1001D800390837193421371D36213A088400380880
:1001E8003921A001A10126080319D829B7182B2104
:1001F8003A08840000083805FF3EA00DA10DB71C81
:100208002B21A60BFA282708371862292008D82995
:100218000830A6003B088400390837193421371DF7
:1002280036213A08840038093D2126080319D829BF
:10023800371862213A088400A10CA00C0008380481
:10024800031C380680002B21A60B1E29D8293B0841
:100258008400390880060000312932298006080008
:1002680080043C29FF3A80053D2984178004D82959
:10027800FF3A84178005D829A301A200FF30A207FE
:10028800031CA307031CD8290330A100E4304E2126
:100298004229A101F63EA000A109031C5929FE30FC
:1002A8000000A00703185429A0076400A10F5329D0
:1002B800000020185F29201861290800A201A30165
:1002C8006929A10CA00CA20DA30DFF3E03186529F6
:1002D8002308A1002208A000D829A20002307F2903
:1002E800A20003307F29A20001307F29A200063036
:1002F8007F29A2000530A80023082102031D8629B2
:10030800220820020430031801300319023028059E
:10031800031DFF30D8290404031DFF30D829A2008B
:100328002008A6002408A0002608A4002108A6008A
:100338002508A1002608A500A329A501A4011030BD
:10034800A600210DA40DA50D2208A4022308031C54
:10035800230FA5020318B7292208A40723080318A6
:10036800230FA5070310A00DA10DA60BA529200892
:10037800D8291030A800A101A001A70CA60C031CC5
:10038800CB292208A00723080318230FA107A10CD3
:10039800A00CA50CA40CA80BC1292408D8298400FA
:1003A80031088A0030088200831303138312640023
:1003B8000800831607309F00AA01AB01A801A90114
:1003C8008312DA01DB01D801D901E201E301E0017E
:1003D800E1018316D201D6018613061386129030E6
:1003E80087000710871007118716D3018312CC01E5
:1003F800CD018316D801AE01AF018312C601C70132
:10040800F401F501BC01BD010130A300F4308A01FB
:100418004121861383168613831286128316861249
:10042800831206138316061307308312BA0040306E
:10043800B8002030AA00AB01AE01AF0153308A01E9
:10044800692074308A01692061308A01692072301C
:100458008A01692074308A01692069308A0169201B
:100468006E308A01692067308A0169202E308A013E
:1004780069202E308A0169202E308A0169202E30A9
:100488008A0169200A308A0169200D308A016920B1
:100498008A110A16A72A07148316FF30D1000A30DA
:1004A800CF0083128A110A120D25071032308A01F3
:1004B800402183164030CE009530D0008312831639
:1004C8004E08D10007308312BA000230B800073056
:1004D800BB000430B9000130B700831651088312FD
:1004E800A000A1018A010C218316D1010430CF009C
:1004F80083128A110A120D2583165008D10007307D
:100508008312BA000230B8000730BB000430B900CB
:100518000130B700831651088312A000A1018A0197
:100528000C2183160130CD0083128A110A12292367
:10053800071432308A0140210710640083165908D5
:10054800003C8A110A1283120319ED2A0714831634
:10055800FF30D10007308312BA000230B8000730EC
:10056800BB000430B9000130B7008316510883126C
:10057800A000A1018A010C218A110A1289250710FD
:1005880083164130D10007308312BA000230B80018
:100598000730BB000430B9000130B700831651089A
:1005A8008312A000A1018A010C218316D101043015
:1005B800CF0083128A110A120D258316FF30D1004D
:1005C80083128A110A1266258A110A1289258A015C
:1005D800A12A8316FF30D10007308312BA004030B9
:1005E800B8002030AA00AB01AE01AF014D308A013E
:1005F80069204D308A01692043308A016920203002
:100608008A01692049308A0169204E308A016920AF
:1006180049308A01692054308A01692020308A01D2
:1006280069204F308A0169204B308A0169202130C6
:100638008A0169200A308A0169200D308A016920FF
:1006480086168316861283120800640083165908DA
:100658004D028A110A1283120319422B0730BA007D
:100668002030B8000730BB000430B900B7018A0158
:10067800E7208316D90083128A01292B08008617E0
:1006880083168613831207148316FF30CC00831257
:100698008A110A1277258A110A12892507108316EA
:1006A8005830C80083123F088316C90083123E08D9
:1006B8008316CA00831241088316CB0083124008B0
:1006C8008316CC0083128A110A1233258316FF3051
:1006D800CC0083128A110A1277258A110A128925F9
:1006E8008316CD0183128A0129238316FE30CC009C
:1006F80083128A110A1277254E08BC004F08BD00E4
:100708003C08A0003D08A1005108A30050088A0138
:1007180077218A110A12031DBF2B0730BA00103047
:10072800B8000730BB000830B900A0308A011F208C
:100738003D088A011F203C088A011F208A010420E5
:100748008316D10007308312BA000230B800073090
:10075800BB000430B9000130B7008316510883127A
:10076800A000A1018A010C21BC0A0319BD0A8A1143
:100778000A12031D842B8316FF30D1000230CF00EC
:1007880083128A110A120D258A110A1289250F303F
:1007980083165905DC0083128A110A128925640020
:1007A80083165908003C8A110A128312031DEC2B88
:1007B8000730BA002030B8000730BB000430B90059
:1007C800B7018A01E7208316D90083128A01D32B47
:1007D8008A110A12C7248613831686138312080007
:1007E80007148316FF30CC0083128A110A1277256A
:1007F8008A110A128925071083165130C8008312FE
:100808003F088316C90083123E088316CA00831264
:1008180041088316CB00831240088316CC0083124C
:100828008A110A1233258316FF30CC0083128A11ED
:100838000A1277258A110A1289258316CD01831297
:100848008A0129238316FE30CD0083128A012923C9
:100858004E08CA004F08CB004A08A0004B08A10068
:100868005108A30050088A0177218A110A12031D32
:10087800682C0730BA002030B8000730BB000430BD
:10088800B900B7018A01E7208316D1000730831227
:10089800BA001030B8000730BB000830B900A030EB
:1008A8008A011F204B088A011F204A088A011F203D
:1008B8008316510883128A011D20CA0A0319CB0A1C
:1008C8008A110A12031D302C8A110A1289258A11ED
:1008D8000A1289258A110A12C72408008316503083
:1008E800CE0083128A110A129224080083166030FF
:1008F800CE0083128A110A129224080083166130EE
:10090800CE0083128A110A129224080083166630D8
:10091800CE0083128A110A12922408000714831643
:10092800FF30CC0083128A110A1277258A110A1225
:100938008925071083164E08C80083123F088316BE
:10094800C90083123E088316CA0083124108831621
:10095800CB00831240088316CC0083128A110A1236
:1009680033258316FF30D1000230CF0083128A115D
:100978000A120D258A110A1289258316CD018312C0
:100988008A012923080007148316FF30D100073095
:100998008312BA000230B8000730BB000430B90037
:1009A8000130B700831651088312A000A1018A0103
:1009B8000C218A110A128925071083164D30CC00A4
:1009C80083128A110A1277258316D1010430CF00C9
:1009D80083128A110A120D258316FF30CC00831268
:1009E8008A110A1277250730BA002030B80007307C
:1009F800BB000430B900B70110308A01E820831623
:100A0800A600831221088316A7002608D80083129F
:100A1800080083160130DC008312640083165C082A
:100A28004F028A110A128312031C322D0730BA00B2
:100A38000230B8000730BB000430B9000130B700FD
:100A4800831651088312A000A1018A010C21831684
:100A5800DC0A8A110A128312031D112D08000730BF
:100A6800BA000230B8000730BB000430B9000130CA
:100A7800B700831648088312A000A1018A010C213F
:100A88000730BA000230B8000730BB000430B900A4
:100A98000130B700831649088312A000A1018A011A
:100AA8000C210730BA000230B8000730BB00043010
:100AB800B9000130B70083164A088312A000A101CB
:100AC8008A010C210730BA000230B8000730BB0099
:100AD8000430B9000130B70083164B088312A00018
:100AE800A1018A010C210730BA000230B800073092
:100AF800BB000430B9000130B70083164C088312DC
:100B0800A000A1018A010C2108000730BA0020309A
:100B1800B8000730BB000430B900B7018A01E720EC
:100B28008316D90083120800CE010830CF00FF30A9
:100B3800D0000930D100BE01BF01C001C1018A0146
:100B4800F4230B30BC000830BD000730BA00103069
:100B5800B8000730BB000830B900A0308A011F2058
:100B68003D088A011F203C088A011F208A010420B1
:100B7800C4000C30BC000830BD000730BA0010308B
:100B8800B8000730BB000830B900A0308A011F2028
:100B98003D088A011F203C088A011F208A01042081
:100BA800C5000D30BC000830BD000730BA00103059
:100BB800B8000730BB000830B900A0308A011F20F8
:100BC8003D088A011F203C088A011F208A01042051
:100BD8008316DA0083120E30BC000830BD000730DF
:100BE800BA001030B8000730BB000830B900A03098
:100BF8008A011F203D088A011F203C088A011F2006
:100C08008A0104208316AC0083120F30BC00083020
:100C1800BD000730BA001030B8000730BB000830FC
:100C2800B900A0308A011F203D088A011F203C0816
:100C38008A011F208A0104208316AD008312113017
:100C4800BC000830BD000730BA001030B8000730CB
:100C5800BB000830B900A0308A011F203D088A0176
:100C68001F203C088A011F208A0104208316A40043
:100C780083121230BC000830BD000730BA001030B3
:100C8800B8000730BB000830B900A0308A011F2027
:100C98003D088A011F203C088A011F208A01042080
:100CA8008316A50083121630BC000830BD0007303B
:100CB800BA001030B8000730BB000830B900A030C7
:100CC8008A011F203D088A011F203C088A011F2035
:100CD8008A010420F6001730BC000830BD00073038
:100CE800BA001030B8000730BB000830B900A03097
:100CF8008A011F203D088A011F203C088A011F2005
:100D08008A010420F7001330BC000830BD0007300A
:100D1800BA001030B8000730BB000830B900A03066
:100D28008A011F203D088A011F203C088A011F20D4
:100D38008A0104208316B80083121430BC000830DE
:100D4800BD000730BA001030B8000730BB000830CB
:100D5800B900A0308A011F203D088A011F203C08E5
:100D68008A011F208A0104208316B900B601B70141
:100D780038088312A000831639088312A100A30142
:100D880000308A017D218A110A12031D332F203079
:100D9800BC000830BD000730BA001030B80007307A
:100DA800BB000830B900A0308A011F203D088A0125
:100DB8001F203C088A011F208A0104208316B800DE
:100DC80083122130BC000830BD000730BA00103053
:100DD800B8000730BB000830B900A0308A011F20D6
:100DE8003D088A011F203C088A011F208A0104202F
:100DF8008316B90083122230BC000830BD000730CA
:100E0800BA001030B8000730BB000830B900A03075
:100E18008A011F203D088A011F203C088A011F20E3
:100E28008A0104208316B60083122330BC000830E0
:100E3800BD000730BA001030B8000730BB000830DA
:100E4800B900A0308A011F203D088A011F203C08F4
:100E58008A011F208A0104208316B7008312831693
:100E680024088312A600831625088312A7002030C1
:100E7800A200A3018A01BD21B2002508B3004408DD
:100E8800B20745080318013EB3070130B20200302B
:100E9800031C013EB3023208A0003308A100440835
:100EA800A2004508A3008A01A1218316A20083128B
:100EB80021088316A30083120230A600A701760832
:100EC800A2007708A3008A01BD21B2002508B3005B
:100ED80083162C088312B20783162D080318013EC7
:100EE8008312B3073208831622078312F8003308E7
:100EF8000318013E831623078312F9007808A60019
:100F08007908A7004408A2004508A3008A01BD216A
:100F1800FC002508FD007808A6007908A700440809
:100F2800A2004508A3008A01BD212008FA00210873
:100F3800FB007A08D4007B08D5007C08D6007D0821
:100F4800D700D801D9014408A6004508A700831690
:100F58002C088312A20083162D088312A3008A018D
:100F6800BD21DA002508DB007608A6007708A7006F
:100F7800A2010230A3008A01BD21E2002508E30096
:100F88007608A6007708A700A2010230A3008A010C
:100F9800BD212008E0002108E1005A08E2075B08AB
:100FA8000318013EE30764008A110A12031CDF2FAD
:100FB800E00A0319E10A7608A6007708A700A2014B
:100FC8000230A3008A01BD2120088316A8008312DD
:100FD80021088316A90083127608A6007708A700BF
:100FE800A2010230A3008A01BD218316AA00831240
:100FF80025088316AB00831260088316A80783129E
:1010080061080318013E8316A90783126208831634
:10101800AA07831263080318013E8316AB0764000E
:101028008A150A128312031C1E288316A80A03199C
:10103800A90A8312831636088312A000831637087C
:101048008312A100A30100308A017A218A150A12AD
:10105800031D31288A150A12632878088316380276
:10106800B20083127908031C013E83163902B300CB
:1010780032088312A000831633088312A100831656
:101088005A088312A200A3018A01A1218316B20083
:10109800831221088316B30032088312A000831636
:1010A80033088312A1000F30A300F5308A017421A0
:1010B8008A150A12031D63288A110A16202B831623
:1010C8001030D500831283165A088312A600A70190
:1010D8004408A2004508A3008A01BD21C8002508CC
:1010E800C9000800CE010230CF00FF30D000033025
:1010F800D100831628088312BE008316290883129C
:10110800BF0083162A088312C00083162B08831297
:10111800C1008A01F4230730BA001030B800073044
:10112800BB000830B900A0308A011F2002308A01B4
:101138001F203F308A011F208A010420FF0007304A
:10114800BA001030B8000730BB000830B900A03032
:101158008A011F2002308A011F203E308A011F2089
:101168008A010420FE000730BA001030B8000730AA
:10117800BB000830B900A0308A011F2002308A0164
:101188001F203D308A011F208A0104208316A100F8
:1011980007308312BA001030B8000730BB0008309F
:1011A800B900A0308A011F2002308A011F203C307C
:1011B8008A011F208A0104208316A00007308312A9
:1011C800BA001030B8000730BB000830B900A030B2
:1011D8008A011F2002308A011F203B308A011F200C
:1011E8008A0104208316B10007308312BA00103038
:1011F800B8000730BB000830B900A0308A011F20B2
:1012080002308A011F203A308A011F208A010420F7
:101218008316B00083127E088316BE0083127F08EF
:101228008316BF002008C0002108C10083124808A7
:101238008316BC00831249088316BD0083128A15E1
:101248000A1244270230831644078312D2008316F9
:1012580045080318013E8312D30083163008831211
:10126800A000831631088312A100A30100308A016F
:101278007D218A150A12031D742983160230B000D5
:10128800B10107308312BA001030B8000730BB0034
:101298000830B900A0308A011F2002308A011F20BF
:1012A8003B308A011F208316310883128A011D20D2
:1012B8000730BA001030B8000730BB000830B9005A
:1012C800A0308A011F2002308A011F203A308A018B
:1012D8001F208316300883128A011D20C601C7010A
:1012E8007E08D4007F08D500831620088312D60014
:1012F800831621088312D7007C08D6077D080318B7
:10130800013ED70764008A150A12031C8E29D40AE5
:101318000319D50A831620088312A0008316210812
:101328008312A100A30100308A017721B2007E0850
:10133800A0007F08A100A30100308A017721B40032
:101348003208840034088A018F21B400B500640093
:10135800340835048A150A120319D1297E08831620
:10136800BE0083127F088316BF002008C000210832
:10137800C100831248088316BC00831249088316EB
:10138800BD0083128A150A12442783164208831265
:10139800C600831643088312C7008A150A12422220
:1013A80083162C0883127402B20083162D08031CBE
:1013B800013E83127502B3003208A0003308A10071
:1013C8000330A200A3018A01A12124088316DB00AF
:1013D8005B0883127402B2007508031CFF3EB30059
:1013E8003208A6003308A7004408A2004508A30055
:1013F8008A01BD21DE002508DF0083165B08831201
:101408007402B2007508031CFF3EB3003208A60040
:101418003308A7004408A2004508A3008A01BD219B
:101428002008DC002108DD007608A6007708A70060
:101438004408A2004508A3008A01BD21E60025084A
:10144800E7007608A6007708A7004408A200450828
:10145800A3008A01BD212008E4002108E5005E08F8
:10146800E6075F080318013EE70764008A150A12B9
:10147800031C412AE40A0319E50A080064008316DC
:1014880055080C3C8A150A128312031D772A03108B
:10149800530CEF00520CEE005208EE0753080318E5
:1014A800013EEF0764008A150A12031C612A013005
:1014B800EC00ED018A150A12632AEC01ED015208CD
:1014C800A6005308A7000330A200A3018A01BD218A
:1014D800B2002508B3000310330CEB00320CEA000D
:1014E8008A150A12942A5208A6005308A700023047
:1014F800A200A3018A01BD21EE002508EF005208D1
:10150800A6005308A7000230A200A3018A01BD214A
:101518002008EC002108ED006E08EA006F08EB00D7
:101528006A08A0006B08A100A2010630A3008A0186
:10153800A1212408CC002508CD006C088316BE0024
:1015480083126D088316BF0083126E088316C000CD
:1015580083126F088316C100831244088316BC00E7
:10156800831245088316BD0083128A150A12442780
:10157800831644082C078312F400831645080318C1
:10158800013E2D078312F5007408A6007508A70010
:101598004408A2004508A3008A01BD21DA002508F5
:1015A800DB007408A6007508A7004408A2004508D7
:1015B800A3008A01BD212008D8002108D900760897
:1015C800A6007708A7004408A2004508A3008A01DE
:1015D800BD21E2002508E3007608A6007708A700E9
:1015E8004408A2004508A3008A01BD212008E000A4
:1015F8002108E1005A08E2075B080318013EE307E7
:1016080064008A150A12031C0C2BE00A0319E10A6C
:101618000800CE011030CF00FF30D0001130D100CB
:101628005C08BE005D08BF005E08C0005F08C1001E
:101638008A01F423CE011230CF00FF30D0001330DE
:10164800D1000030C00702300318013EC107640012
:101658008A150A12031C332BBE0A0319BF0A8A0112
:10166800F423CE011430CF00FF30D0001530D10064
:1016780000305E07C00004300318013E5F07C10058
:1016880064008A150A12031C4C2BBE0A0319BF0AF0
:101698008A01F423080083165030CE008312BE015D
:1016A800BF014208C0004308C1008A019224080013
:1016B8005608A0005708A100FF30A300FF308A0198
:1016C8007D218A150A12031D712BD40A0319D50A24
:1016D800D601D7018A150A12742BD60A0319D70A1C
:1016E8000800831620088312A0008316210883129D
:1016F800A100FF30A300FF308A017D218A150A125C
:10170800031D902BFE0A0319FF0A8316A001A101ED
:1017180083128A150A12952B8316A00A0319A10AA7
:10172800831208000730BA001030B8000730BB0039
:101738000830B900A0308A011F2083162F088312B1
:101748008A011F2083162E0883128A011F20831600
:10175800520883128A011D208316AE0A0319AF0AA4
:101768008312C60A0319C70A8A150A12752346087E
:10177800A0004708A1004908A30048088A017D2164
:101788008A150A12031D0F2C8A150A125B265008A7
:10179800A0005108A1001530A300FF308A017D2167
:1017A8008A150A12031DDC2B83160130D30083121D
:1017B8008A150A12DA24640083165308013C8A1534
:1017C8000A128312031D072C0030DE0706300318A7
:1017D800013EDF0764008A150A12031CF62BDC0A97
:1017E8000319DD0A0030E60706300318013EE70753
:1017F80064008A150A12031C042CE40A0319E50A7A
:101808008A150A120D23D20A0319D30AC601C70181
:101818008316D301831283162E088312A000831621
:101828002F088312A1000230A30000308A017D2115
:101838008A150A12031DBF2C0730BA001030B800F1
:101848000730BB000830B900A0308A011F200230E1
:101858008A011F203F308A011F207F088A011D202E
:101868000730BA001030B8000730BB000830B900A4
:10187800A0308A011F2002308A011F203E308A01D1
:101888001F207E088A011D200730BA001030B800DA
:101898000730BB000830B900A0308A011F20023091
:1018A8008A011F203D308A011F20831621088312D8
:1018B8008A011D200730BA001030B8000730BB007D
:1018C8000830B900A0308A011F2002308A011F2089
:1018D8003C308A011F208316200883128A011D20AC
:1018E80054087A07BE0055080318013E7B07BF005D
:1018F8005608A0005708A100A2010230A3008A01DF
:10190800A1212408B2002508B30032085602C000FD
:101918003308031C013E5702C100CE01CF01FF303E
:10192800D0000130D1008A0143235608A00057088F
:10193800A100FD30A300FF308A017A218A150A121E
:10194800031DB22CD40A0319D50A0030D607023079
:101958000318013ED7078A150A12B82C0030D6079B
:1019680002300318013ED7078316AE01AF01831278
:101978008A150A12C0240800CE010230CF00FF30B9
:10198800D0000330D100831628088312BE008316C6
:1019980029088312BF0083162A088312C000831601
:1019A8002B088312C1008A01432308008A150A12F2
:1019B80042220730BA004030B8002030AA00AB01FC
:1019C800AE01AF0146308A01692061308A01692081
:1019D80074308A01692053308A01692065308A0190
:1019E800692063308A0169203A308A01692004300D
:1019F800A9007408A4007508A5006830B000B101FA
:101A08008A01A62020308A01692046308A0169208F
:101A180061308A01692074308A01692031308A0175
:101A280069203A308A0169200430A9005C08A400C2
:101A38005D08A5006830B000B1018A01A620043015
:101A4800A9005E08A4005F08A5006830B000B101D5
:101A58008A01A62020308A0169204F308A01692036
:101A680066308A01692066308A01692053308A010C
:101A7800692065308A01692074308A0169203A300A
:101A88008A0169200430A9004C08A4004D08A5006B
:101A98006830B000B1018A01A62020308A0169208F
:101AA80045308A01692041308A01692064308A0101
:101AB800692064308A0169200430A9004E08A40016
:101AC8004F08A5006830B000B1018A01A620043093
:101AD800A9005008A4005108A5006830B000B10161
:101AE8008A01A620CE011030CF00FF30D00011307F
:101AF800D1005C08BE005D08BF005E08C0005F083A
:101B0800C1008A0143236408BE006508BF00660857
:101B1800C0006708C1008A0143230730BA0040307B
:101B2800B8002030AA00AB01AE01AF0120308A0115
:101B3800692046308A01692061308A016920743041
:101B48008A01692032308A0169203A308A01692085
:101B58000430A9003E08A4003F08A5006830B00082
:101B6800B1018A01A6200430A9004008A400410858
:101B7800A5006830B000B1018A01A6200D308A01A5
:101B880069200A308A016920CE011230CF00FF3067
:101B9800D0001330D1005C08BE005D08BF000030E3
:101BA8005E07C00002300318013E5F07C1006400F1
:101BB8008A150A12031CE32DBE0A0319BF0A8A01FB
:101BC80043236408BE006508BF0000306607C000F4
:101BD80002300318013E6707C10064008A150A1223
:101BE800031CF92DBE0A0319BF0A8A014323CE013B
:101BF8001430CF00FF30D0001530D1005C08BE0093
:101C08005D08BF0000305E07C00004300318013EC5
:101C18005F07C10064008A150A12031C162EBE0A4B
:101C28000319BF0A8A0143236408BE006508BF0080
:101C380000306607C00004300318013E6707C10082
:101C480064008A150A12031C2C2EBE0A0319BF0A47
:101C58008A0143230800CA011030CB004A08A000BB
:101C68004B08A1001530A300FF308A0177218A159F
:101C78000A12031D5A2E0730BA001030B800073078
:101C8800BB000830B900A0308A011F204B088A0128
:101C98001F204A088A011F2000308A011D20CA0A15
:101CA8000319CB0A8A150A12031D322E080052089E
:101CB800A6005308A7000230A200A3018A01BD2193
:101CC800EA002508EB006A08A0006B08A100A20141
:101CD8000630A3008A01A1212408CC002508CD00E4
:101CE80000304C07CE0010300318013E4D07CF00DE
:101CF80001304E07D0004F080318013ED1005008AC
:101D0800A0005108A1001530A300FF308A017D21F1
:101D18008A150A12031DCA2E013052078316B40011
:101D2800831253080318013E8316B5000730831247
:101D3800BA001030B8000730BB000830B900A03036
:101D48008A011F204F088A011F204E088A011F2080
:101D58008316340883128A011D200730BA00103018
:101D6800B8000730BB000830B900A0308A011F2036
:101D780051088A011F2050088A011F208316350840
:101D880083128A011D208A150A120B2F0730BA0008
:101D98001030B8000730BB000830B900A0308A0105
:101DA8001F204F088A011F204E088A011F20FF307C
:101DB8008A011D200730BA001030B8000730BB0078
:101DC8000830B900A0308A011F2051088A011F205D
:101DD80050088A011F20FF308A011D205208A000E8
:101DE8005308A100A30102308A0171218A150A1241
:101DF800031D432F4E08A0004F08A1001030A30078
:101E080000308A0171218A150A12031D432F0730F9
:101E1800BA001030B8000730BB000830B900A03055
:101E28008A011F2002304E02B2000030031C013E1E
:101E38004F02B30033088A011F2032088A011F208D
:101E480052088A011D200730BA001030B800073048
:101E5800BB000830B900A0308A011F2002305002B0
:101E6800B2000030031C013E5102B30033088A015E
:101E78001F2032088A011F2053088A011D200800EC
:101E880083163E088312A00083163F088312A10020
:101E9800831640088312A400831641088312A50004
:101EA80083163D088312A30083163C0883128A0117
:101EB80093218316C400831221088316C500831258
:101EC80024088316C200831225088316C3008312D0
:101ED80008000800CE01CF01FF30D0000130D1004A
:101EE800BE01BF01C001C1018A014F228A019825A4
:101EF8000730BA004030B8002030AA00AB01AE016C
:101F0800AF010D308A0169200A308A016920423008
:101F18008A01692050308A01692053308A0169207A
:101F28003D308A0169200430A9004408A40045080E
:101F3800A5006830B000B1018A01A6200D308A01E1
:101F480069200A308A0169200730BA004030B80099
:101F58002030AA00AB01AE01AF0153308A016920DD
:101F680050308A01692043308A0169203D308A0156
:101F780069200430A90083165A088312A400A50119
:101F88006830B000B1018A01A6200D308A016920AD
:101F98000A308A0169200730BA004030B800203082
:101FA800AA00AB01AE01AF0152308A01692053305B
:101FB8008A01692043308A0169203D308A016920FD
:101FC8000430A90083162C088312A40083162D0858
:101FD8008312A5006830B000B1018A01A6200D3037
:101FE8008A0169200A308A0169200730BA00403026
:101FF800B8002030AA00AB01AE01AF0152308A010F
:10200800692045308A01692043308A0169203D30C2
:102018008A0169200430A900831624088312A400C9
:10202800831625088312A5006830B000B1018A0123
:10203800A6200D308A0169200A308A0169200730FC
:10204800BA004030B8002030AA00AB01AE01AF01A1
:1020580046308A01692041308A01692054308A015A
:10206800692020308A01692073308A01692065302F
:102078008A01692063308A01692073308A016920E6
:102088003D308A0169200430A9007608A400770849
:10209800A5006830B000B1018A01A6200D308A0180
:1020A80069200A308A0169200730BA004030B80038
:1020B8002030AA00AB01AE01AF0154308A0169207B
:1020C8004F308A01692053308A0169203D308A01E6
:1020D80069200430A900831636088312A4008316E9
:1020E80037088312A5006830B000B1018A01A62024
:1020F8000430A900831638088312A400831639080F
:102108008312A5006830B000B1018A01A6200D3005
:102118008A0169200A308A0169200730BA004030F4
:10212800B8002030AA00AB01AE01AF0152308A01DD
:10213800692044308A01692053308A0169203D3082
:102148008A0169200430A900831622088312A4009A
:10215800831623088312A5006830B000B1018A01F4
:10216800A6200D308A0169200A308A0169200730CB
:10217800BA004030B8002030AA00AB01AE01AF0170
:1021880046308A01692044308A01692053308A0127
:1021980069203D308A0169200430A9007808A4002C
:1021A8007908A5006830B000B1018A01A6200D3079
:1021B8008A0169200A308A0169200730BA00403054
:1021C800B8002030AA00AB01AE01AF0146308A0149
:1021D80069205F308A0169204F308A016920723096
:1021E8008A01692069308A01692067308A0169207B
:1021F8003D308A0169200430A9005408A40055081C
:10220800A5006830B000B1018A01A6200430A900F9
:102218005608A4005708A5006830B000B1018A012B
:10222800A6200D308A0169200A308A01692007300A
:10223800BA004030B8002030AA00AB01AE01AF01AF
:1022480046308A01692041308A01692054308A0168
:10225800692031308A0169205F308A016920613044
:102268008A01692064308A01692064308A01692002
:1022780072308A0169203D308A0169200430A90042
:102288005808A4005908A5006830B000B1018A01B7
:10229800A6200430A9005A08A4005B08A5006830ED
:1022A800B000B1018A01A6200D308A0169200A30E8
:1022B8008A0169200730BA004030B8002030AA00EF
:1022C800AB01AE01AF0146308A01692041308A0175
:1022D800692054308A01692032308A0169205F30D0
:1022E8008A01692061308A01692064308A01692085
:1022F80064308A01692072308A0169203D308A0180
:1023080069200430A9006008A4006108A5006830AD
:10231800B000B1018A01A6200430A9006208A40017
:102328006308A5006830B000B1018A01A6200D300D
:102338008A0169200A308A0169200730BA004030D2
:10234800B8002030AA00AB01AE01AF0152308A01BB
:1023580069206F308A0169206F308A0169207430E2
:102368008A01692044308A01692069308A0169201C
:1023780072308A0169205F308A01692061308A01E0
:10238800692064308A01692064308A0169207230CA
:102398008A0169203D308A0169200430A90083162A
:1023A80028088312A400831629088312A500683020
:1023B800B000B1018A01A6200430A90083162A08BA
:1023C8008312A40083162B088312A5006830B0007E
:1023D800B1018A01A6200D308A0169200A308A01DC
:1023E80069200730BA004030B8002030AA00AB019D
:1023F800AE01AF0143308A0169206C308A0169203F
:1024080075308A01692073308A01692074308A0125
:10241800692065308A01692072308A0169205F303D
:102428008A01692073308A01692069308A0169202C
:102438007A308A01692065308A0169203D308A0135
:1024480069200430A9004808A4004908A50068309C
:10245800B000B1018A01A6200D308A0169200A3036
:102468008A0169200730BA004030B8002030AA003D
:10247800AB01AE01AF0142308A0169204F308A01B9
:1024880069204F308A01692054308A016920203040
:102498008A0169204F308A0169204B308A016920FE
:1024A8000A308A0169200D308A0169208A150A12CA
:1024B80076200730BA004030B8002030AA00AB01BF
:1024C800AE01AF0144308A01692049308A01692090
:1024D80052308A01692020308A0169204F308A01F0
:1024E80069204B308A0169200A308A0169200D3041
:1024F8008A0169208A150A120D230730BA00403074
:10250800B8002030AA00AB01AE01AF0146308A0105
:10251800692041308A01692054308A0169202030BD
:102528008A0169204F308A0169204B308A0169206D
:102538000A308A0169200D308A0169208316AE01AC
:10254800AF01831208008A150A126E270730BA00F5
:102558004030B8002030AA00AB01AE01AF014630D0
:102568008A01692041308A01692054308A01692032
:102578000230A900831655088312A400A50168300B
:10258800B000B1018A01B9200A308A0169200D30F2
:102598008A01692083162130D2000130B200B301CC
:1025A8008312831632088312A0008316330883121D
:1025B800A100A30120308A0177218A110A16031D80
:1025C8001D2B8316C601C701831283164608831282
:1025D800A000831647088312A1000130A300FF3032
:1025E8008A0177218A110A16031D062B8A150A12F9
:1025F80096238316C60A0319C70A8A110A16831274
:10260800031DE92A8316D20A64007F3052028A1118
:102618000A168312031C142B83162130D20083124E
:102628008316B20A0319B30A8A110A168312031D04
:10263800D52A8A110A168C2B0730BA004030B80008
:102648002030AA00AB01AE01AF010A308A0169202F
:102658000D308A01692041308A01692062308A017F
:1026680069206F308A01692072308A0169207430CC
:102678008A01692065308A01692064308A016920ED
:1026880021308A0169200D308A0169200A308A01C7
:10269800692046308A01692041308A016920543016
:1026A8008A01692031308A01692032308A01692023
:1026B80020308A01692063308A01692061308A01EB
:1026C800692072308A01692064308A0169202030CB
:1026D8008A01692064308A01692065308A0169208D
:1026E80074308A01692065308A01692063308A0163
:1026F800692074308A01692065308A016920643054
:102708008A0169200D308A0169200A308A0169200E
:102718000730BA004030B8002030AA00AB01AE0143
:10272800AF010A308A0169200D308A0169204430DE
:102738008A0169204F308A0169204E308A01692058
:1027480045308A01692021308A01692064008A1194
:0C2758000A16AA2B63008A110A16AE2B89
:02400E003D3D36
:00000001FF
